:030000000238E9DA
:0C38E90078FFE4F6D8FD758165023930E7
:1014A40020000A3C2E2E2E3E004950436F6E6E657E
:1014B40063745245510A004950436F6E6E656374FC
:1014C400000A49504E6F41434B210A003E432C56BB
:1014D4002C43432CC0E4E0EFF2E5F020D1E8EDEA40
:1014E400EEEC49500A003E432C4D41432C2530324A
:1014F40062583A25303262583A25303262583A25D9
:10150400303262583A25303262583A2530326258C5
:101514002C4D414320E0E4F0E5F10A003E432C5613
:1015240045522C20332E3220EEF2202573202573D1
:101534002CC2E5F0F1E8FF20495020ECEEE4F3EB97
:10154400FF0A004A756C20303220323030390031C5
:10155400303A31393A3133003E432C4C442C50520A
:101564004F473A2020202020202020202020202007
:101574002020202020202020202020202020202067
:101584002020202020202020202020202020202057
:101594002020202020202020202020202020202047
:1015A40020202020202020202CC4E0F2E020EFF096
:1015B400EEF8E8E2EAE828F4E0E9EB290A003E2A3A
:1015C4002C312CCEF1EDEEE2EDFBE520EFE0F0E086
:1015D400ECE5F2F0FB20F1E5F2E5E2EEE3EE20E8E3
:1015E400EDF2E5F0F4E5E9F1E00A003E412C41308A
:1015F400312C2562752E2562752E2562752E256285
:10160400752C495020E0E4F0E5F120E0E4E0EFF24D
:10161400E5F0E00A003E412C4130322C2562752E63
:101624002562752E2562752E2562752C495020E0A1
:10163400E4F0E5F120EEF1ED2E20F1E5F0E2E5F045
:10164400E00A003E412C4130332C2562752E256280
:10165400752E2562752E2562752C495020E0E4F024
:10166400E5F120F0E5E72E20F1E5F0E2E5F0E00A0F
:10167400003E412C4130342C2562752E2562752E96
:101684002562752E2562752CCCE0F1EAE020F1E5A7
:10169400F2E80A003E412C4130352C2562752E2596
:1016A40062752E2562752E2562752CD8EBFEE70A2D
:1016B400003E2A2C312CC4EEEF2E20EFE0F0E0ECBB
:1016C400E5F2F0FB20F1E5F2E5E2EEE3EE20E8EDF1
:1016D400F2E5F0F4E5E9F1E00A003E422C53303142
:1016E4002C2562752CC6E4E0F2FC20E7E0EFF0EE76
:1016F400F1E020F1EEE5E4E8EDE5EDE8FF20EEF2BF
:1017040020F1E5F0E2E5F0E00A003E422C533032ED
:101714002C2562752CCEE1ECE5ED20F120F1E5F00D
:10172400E2E5F0EEEC20E1E5E720EAE2E8F2E0EDC4
:10173400F6E8E90A003E422C5330332C2562752C1E
:10174400CFE5F0E5E7E0EFF3F1EA20EFF0E820EF92
:10175400EEF2E5F0E520F1E2FFE7E820F120F1E523
:10176400F0E2E5F0EEEC0A003E454E440A000A447D
:10177400756D7058202020202030302030312030EA
:10178400322030332030342030352030362030378A
:10179400203038203039203041203042203043205E
:1017A4003044203045203046000A3A003A20000AEE
:1017B400000A44756D7044202020202030302030F1
:1017C4003120303220303320303420303520303650
:1017D400203037203038203039203041203042202A
:1017E400304320304420304520304600457272207A
:1017F4006B657900526420656570726F6D0A0052E2
:1018040064204D454D0A00526420436F64650A000C
:10181400577269746520436F64650A004465627594
:10182400674950204F4E0A0044656275674950204D
:101834004F46460A00446562756755736572204FCA
:101844006E0A00446562756755736572204F46469B
:101854000A0044656275674D7367204F6E0A004441
:10186400656275674D7367204F46460A00436F6E85
:10187400666967206C6F636B210A00577220656587
:1018840070726F6D0A002053617665206565707211
:101894006F6D210A00457272204D414321004C6F47
:1018A40061643E3E002A00CEF8E8E1EAE00A002046
:1018B4002D202575282575290A003C4130313D002D
:1018C4003C4130323D003C4130333D003C413034FA
:1018D4003D003C4130353D003C21003C5330313D1E
:1018E400003C5330323D003C5330333D003C5330D8
:0918F400353D003C5330363D0047
:06430400010B000109009D
:1042F400C28E438910758BFF758DB7D2ABD28E22D7
:03001B000237CBDE
:1037CB00C0E0C083C082C0D0C28E758BFF758DB731
:1037DB0020060675A61E75A6E10509D202E50B604B
:1037EB0002050BE50AD394014002150A050EE50EFE
:1037FB00540F7048D20EE50E543F7012D2009066F3
:10380B008DE0600A04F0E0D394B44002D2069066D7
:10381B0086E0600204F0906104E0600214F09066B0
:10382B008EE0D394014003E014F0300502050CE563
:10383B000DD394644004D2068002050DE508D394A1
:10384B000140021508D28ED0D0D082D083D0E03286
:1008D000C291C290D2B5C20B7D027C007F0712424A
:1008E000BD8F47E547646060097D017F6012425813
:1008F000D20BE4FDFC7F0B1242BD8F47E54730E68B
:10090000097D04E4FF12427CD20B7D017C007F074D
:100910001242BD8F47E5477008FD7FFF124258D253
:100920000B300B03126000C288C2A8C2AA758900EE
:10093000123C9690633EE0B4FA06A3E064CE607B7E
:10094000E4F54774362547F582E43463F583E4F033
:100950000547E547B443EC90633E74FAF0A374CEC8
:10096000F0A374CCF0906344740AF0E4A3F0A30401
:10097000F0A3F090633A74FFF0A3F0A3F0E4A3F0C7
:10098000906355740AF0E4F547E5472401FFE4332A
:10099000FE74362547F582E43463F583E0FD1242A8
:1009A000340547E547C3944340DFE4F5A775A61E29
:1009B00075A6E1907FF0F0A3F080FE906349740388
:1009C000F0A374CCF0E4906348F090668BF0A3F051
:1009D0001234DFC2B5123668C2061240BCD20BC256
:1009E0000DC20C9065767408F09062B47424F0E443
:1009F000A3F090633EE09062B6F090633FE09062B7
:100A0000B7F0906340E09062B8F0906341E090628C
:100A1000B9F0906342E09062BAF0906343E0906274
:100A2000BBF0750A01E4906577F0C207C208C209FD
:100A3000C20A200B18AF47FE7D03123247E4FF12B3
:100A4000371B7E147FA4E4FBFDFC122E6490668DA0
:100A5000E060037401F0E4906104F0F50C906575BA
:100A6000F0F50D1242F475A70775A61E75A6E1D222
:100A7000AFE4F50D906104E07003120F3F90668EB5
:100A8000E06401701D9080007410F09080A874FFE5
:100A9000F0A3F0A3F0A3F0E490668EF0D20BC20CAA
:100AA000C20D908008E0F54730E405D2077410F0DD
:100AB000E54730E508D2099080087420F0E547301A
:100AC000E608D2089080087440F0E50CC394034017
:100AD00019908002E4F0908001F0908000F0E50C25
:100AE00094064006E4F50C1240BC9080A0E0700330
:100AF000123E069080B8E07003123D149080D0E062
:100B00007003124060908000E07013300710122FC5
:100B10006B906331EFF0D394004003120026908075
:100B200002E07006908000E06005D205020A71C202
:100B300005E4F50C906104E06003020A71200B12D9
:100B4000906578E0600C7E147FA612315FE49065BA
:100B500078F0300912122AA7906331EFF0D3940095
:100B60004005E0FF120022200803020CE7122920B2
:100B7000906331EFF07003020A71906375E054BF27
:100B8000247F7003020C50147003020C28240260AE
:100B900003020C89200B077E147FAD12315F200FFA
:100BA00003020CE790634DE07006906351E06067CC
:100BB000906682E0FF90634DE0B50724906683E085
:100BC000FE90634EE0B50618906684E0FE90634F99
:100BD000E0B5060C906685E0FE906350E06E6037ED
:100BE000906351E06F6003020CE7906683E0FF9032
:100BF0006352E06F6003020CE7906684E0FF90634D
:100C000053E06F6003020CE7906685E0FF90635449
:100C1000E06F6003020CE7C2039065777401F01285
:100C2000430E750A01020CE790668DE060037401C3
:100C3000F090667AE0FF906377E06F6003020CE764
:100C400090667AE004F0E4F50A906575F0020CE72E
:100C5000300303020CE7906344E07003020A7190D2
:100C60006355740AF012430CD203E4F50A906575DB
:100C7000F090668604F0E4906679F0A3F0200B67AC
:100C80007E147FBB12315F805E90668DE0600374DE
:100C900001F0300352906375E020E74B906377E0FA
:100CA000FF906679E0FE6F600D906681E07007EE60
:100CB000146F70338013906679E004F0906331E034
:100CC000FFD39404400312430D9060007482F0A39C
:100CD0007401F0906377E0906002F07E607F007DA9
:100CE000031239FC020A71200303020DFFE50A70AA
:100CF0006812385BEF60237E647F75906476E02431
:100D000004FD1239FC906681E07009906355E0F5AE
:100D10000A020A71E4F50A020A71906686E0D39429
:100D20003C4036906681E0703090668604F0124355
:100D30000BE4906475F0A37412F090667AE090640E
:100D400077F0A374FDF090610563A201906479636C
:100D5000A2017F1212266E809E12001E8F47E54769
:100D6000B401159060007483F0E4A3F07E607F000E
:100D70007D021239FC020A71E547D39401401C90B0
:100D800060007483F0A37401F0E54724FEA3F07EB5
:100D9000607F007D031239FC020A71E50A6401607C
:100DA00003020A71906575E004F0200B077E147F42
:100DB000C512315F906355E0C394C85004E02432FB
:100DC000F0906575E0C39405400DC203E49065772B
:100DD000F012430E020A717C667D82906349E0FA4C
:100DE000A3E0FB7F02123C127E647F75906476E084
:100DF0002404FD1239FC906355E0F50A020A71E5FE
:100E00000A64016003020A71906577E01460462469
:100E1000FE6042147003020EF224046003020A71A1
:100E2000E4F50C200F139065777404F0906575E07D
:100E30005401F0750A01020A719080027410F0E406
:100E4000906577F090657504F0750AFA9066827483
:100E5000FFF0020A71906682E07003020EDC90647B
:100E6000757480F09064777401F0E4A3F0A304F04B
:100E7000A37430F0A3747BF0E4F547747C2547F548
:100E800082E43464F583747DF0747D2547F582E453
:100E90003464F583E4F0E5472407906476F07C66DB
:100EA0007D82906349E0FAA3E0FB7F02123C127E50
:100EB000647F75E5472409FD1239FC906681E06086
:100EC0001B12430CD203E4F50A906575F090668618
:100ED00004F0E4906679F0A3F0020A71300F07E4A1
:100EE000906577F080069065777404F0750AFA02D1
:100EF0000A719080027410F0750A05906575E064BF
:100F000001FFF09065777401F0EF7019906351E084
:100F10006013FCA3E0FDA3E0FEA3E0FF9066821255
:100F20002241020A7190634DE0FCA3E0FDA3E0FEC4
:0E0F3000A3E0FF906682122241020A7180FE49
:010F3E002290
:10002600906376E0B444047F0180027F009063759C
:10003600E0B447047E0180027E00EE5F604A906372
:100046003EE0906377F090633FE0906378F09063D2
:1000560040E0906379F0906341E090637AF09063BA
:1000660042E090637BF0906343E090637CF09063A2
:10007600767452F09062AE63A2019080A863A201EA
:100086007F0612266E0208C6906331E0C3940850BC
:10009600030208CF90633EE0FF906377E06F600352
:1000A6000208CF90633FE0FF906378E06F60030241
:1000B60008CF906340E0FF906379E06F6003020829
:1000C600CF906341E0FF90637AE06F60030208CF50
:1000D600906342E0FF90637BE06F60030208CF907D
:1000E6006343E0FF90637CE06F60030208CF906398
:1000F60076E06444701A9080A8E0B4FF139062AE74
:1001060063A2019080A863A2017F0612266E80106A
:100116009062B2E09080ACF09062B3E09080ADF077
:1001260090668DE060037401F090668E7464F090C2
:1001360063767452F0906375E0646D600302026941
:100146007BFF7A1479D0121D697BFF7A1479EA90C5
:10015600633EE0F550A3E0F551A3E0F552A3E0F5C8
:1001660053A3E0F554A3E0F555121D697550FF75CC
:1001760051157552477553FF7554157555537BFFC9
:100186007A157920121D697BFF7A15795C121D6933
:100196007BFF7A1579C2121D697BFF7A1579EF907C
:1001A6006344E0F550A3E0F551A3E0F552A3E0F572
:1001B60053121D697BFF7A16791990634DE0F5504D
:1001C600A3E0F551A3E0F552A3E0F553121D697BB8
:1001D600FF7A167947906351E0F550A3E0F551A3F5
:1001E600E0F552A3E0F553121D697BFF7A16797587
:1001F60090633AE0F550A3E0F551A3E0F552A3E091
:10020600F553121D697BFF7A167998906336E0F5EF
:1002160050A3E0F551A3E0F552A3E0F553121D6992
:100226007BFF7A1679B5121D697BFF7A1679DEA2F5
:100236000FE433F550121D697BFF7A17790E90662D
:1002460081E0F550121D697BFF7A17793990668D2A
:10025600E0F550121D69122C187BFF7A17796C1283
:100266001D6922906375E0644C70737E177F72FB84
:10027600FDFC122E6490637DE0F548A3E0F549E4A9
:10028600F54BE54890637FF0A3E549F07E177FAD17
:100296007C637D7F7B02122E64E4F54A8549828564
:1002A6004883E0FF747F254AF582E43463F583EFE3
:1002B600F00549E54970020548054AE54AB410DCEF
:1002C6007E177FB07C637D7F7B10122E64054BE525
:1002D6004BC3941040AC7E177FB312315F229063FC
:1002E60075E0646C7060F54C7E177FB5FBFDFC1203
:1002F6002E64E4F54BE490637FF0A3E54CF07E17A3
:100306007FAD7C637D7F7B02122E64E4F54AA84CA8
:10031600E6FF747F254AF582E43463F583EFF00542
:100326004C054AE54AB410E67E177FB07C637D7FB4
:100336007B10122E64054BE54BC3940840B77E171D
:100346007FB312315F22906375E0644B7061F54AAA
:100356007467254AF582E43463F583E06032746796
:10036600254AF582E43463F583E0F4602374672557
:100376004AF582E43463F583E0FF747D254AF5820D
:10038600E43463F583E0B50710054AE54AB408C0CE
:100396009061047432F00208C69063757421F030DF
:1003A6000B030208C67E177FF012315F0208C69063
:1003B6006375E0B4521A200B077E177FF812315F7F
:1003C6009063757472F07E637F757D0812397522AD
:1003D600906375E064497045200B077E187F031211
:1003E600315F90637DE0F548A3E0F549E4F54A8581
:1003F6004982854883E0FF747F254AF582E43463A9
:10040600F583EFF00549E54970020548054AE54AD6
:10041600B480DC7E637F757D8A12397522906375A0
:10042600E064437046200B077E187F0B12315F9005
:10043600637DE0F548A3E0F549E4F54A8549828500
:100446004883E493FF747F254AF582E43463F58399
:10045600EFF00549E54970020548054AE54AB480CA
:10046600DB7E637F757D8A12397522906375E06441
:100476005A7053200B077E187F1412315F90637DEC
:10048600E0F548A3E0F5497C637D7F7B80AF49AE0C
:10049600481241DAE4F54A854982854883E493FFA8
:1004A600747F254AF582E43463F583EFF00549E568
:1004B6004970020548054AE54AB480DB7E637F75CC
:1004C6007D8A12397522906375E0644460030205E3
:1004D6005D90637DE0FF644470030208C6EFB431AB
:1004E6000CC20B7E187F2012315F0208C690637D16
:1004F600E0B4300CD20B7E187F2C12315F0208C696
:1005060090637DE0B4320CD20C7E187F3912315FD5
:100516000208C690637DE0B4330CC20C7E187F4798
:1005260012315F0208C690637DE0B4340CD20D7EB2
:10053600187F5612315F0208C690637DE0B4350C11
:10054600C20D7E187F6312315F0208C690637DE09C
:10055600FF1200210208C6906104E07013200B0709
:100566007E187F7112315F9063757421F00208C6A0
:100576009061047432F0906375E0FFB45104C2AF29
:1005860080FEEF64577045200B077E187F7F12317F
:100596005F90637EE0906331F0E4F54A906331E06A
:1005A600FFE54AC39F40030208C6747F254AF582C9
:1005B600E43463F583E0FF90637DE0254A24ADF5DE
:1005C60082E43461F583EFF0054A80D0906375E0EC
:1005D60064536003020680200B077E187F8A12315F
:1005E6005F90633EE0FF9061B6E06F703C90633FC2
:1005F600E0FF9061B7E06F7030906340E0FF90617C
:10060600B8E0B50724906341E0FF9061B9E0B50713
:1006160018906342E0FF9061BAE0B5070C9063431F
:10062600E0FF9061BBE06F60169063757421F03057
:100636000B030208C67E187F9912315F0208C6E4D2
:10064600F54AE4F50DAF4AFE74AD254AF582E43469
:1006560061F583E0FD124234054AE54AC394FE4043
:10066600E1C2AFE4907FF0F0A3F0907FFD74AAF0B2
:10067600A374FFF0A37455F080FE906375E0644F99
:10068600705A90637DE0F548A3E0F549E549454891
:10069600700A200B077E187FA212315F200B077E9F
:1006A600187FA912315FE4F54A747F254AF582E482
:1006B6003463F583E0854982854883F00549E54939
:1006C60070020548054AE54AB480DE90668CE0244F
:1006D60080F090668BE03400F00208C6906375E007
:1006E6006445707490637DE0FEA3E0FF907FF0EEBA
:1006F600F0A3EFF0D39400EE94044038907FF0E03E
:10070600FEA3E0FF90668BE0FCA3E0FD9FEC9E401D
:1007160023E42FFFEE3401FED3ED9FEC9E5015C26D
:10072600AF907FFD74AAF0A374FFF0A37455F0E4B4
:10073600F5A780FE7E187FAB12315F7BFF7A1879B2
:10074600B3907FF0E0F550A3E0F55190668BE0F5AD
:1007560052A3E0F553121D69906375E0646560036A
:100766000208CF90637DE0FFA3E0907FF0CFF0A377
:10077600EFF0E4F548F549D3907FF1E09549907F95
:10078600F0E095484020E4F50D2549FFE5483401A1
:10079600FE854982854883E0FD1242340549E549D4
:1007A6007002054880D17E187FBE123A83EF4E60F4
:1007B60020120003906344EFF0120003906345EFAC
:1007C600F0120003906346EFF0120003906347EFC8
:1007D600F07E187FC4123A83EF4E60201200039019
:1007E600634DEFF012000390634EEFF0120003909A
:1007F600634FEFF0120003906350EFF07E187FCA4C
:10080600123A83EF4E6020120003906351EFF0120C
:100816000003906352EFF0120003906353EFF0125F
:100826000003906354EFF07E187FD0123A83EF4EA8
:10083600602012000390633AEFF012000390633BCE
:10084600EFF012000390633CEFF012000390633D5B
:10085600EFF07E187FD6123A83EF4E602012000327
:10086600906336EFF0120003906337EFF012000347
:10087600906338EFF0120003906339EFF0E4F54A25
:10088600E4F50DE54A2401FFE433FE7436254AF506
:1008960082E43463F583E0FD124234054AE54AC337
:1008A600944340DCC2AFE4907FF0F0A3F0907FFD6C
:1008B60074AAF0A374FFF0A37455F0E4F5A780FEC4
:0908C6007E637F757D081239750F
:0108CF002206
:1041A200AE07EEC39430400BEED394395005EE24A3
:1041B200D0FF22EEC39461400BEED394665005EE1D
:1041C20024A9FF22EEC39441400BEED3944650053E
:0841D200EE24C9FF22AF062212
:1042DA009062ADE004F070069062ACE004F0906287
:0A42EA00ACE0FEA3E0FF1242A022A8
:100003001242DA1241A2EFC454F0FEC0061242DAE1
:080013001241A2D0E02FFF22F0
:10400300E4906B5FF01242DA906B60EFF0C3943090
:104013004018E0FFD394395011906B5FE02405F50D
:1040230082E43461F583EFF08011906B5FE0240547
:10403300F582E43461F583E4F0800C906B5FE00477
:10404300F0E0D3940840BE754D00754E00754F00E7
:0C405300E4F5507B017A61790512277CAE
:01405F00223E
:043A83008E4D8F4E87
:103A87009062ACE4F0A374FFF01242DAEF606EF4D8
:103A9700606B854E82854D83E493B507EC754F01C6
:103AA700E54E254FF582E4354DF583E49360259087
:103AB70062ADE0254FFF9062ACE03400FE1242A0F9
:103AC700E54E254FF582E4354DF583E493B50704BC
:103AD700054F80CCE54E254FF582E4354DF583E45F
:103AE7009370A6E54F24FFFFE434FFFE9062ADE03C
:103AF7002FF09062ACE03EF07E007F0122E4FEFFF3
:013B0700229B
:1034DF007E187FDC123A83EF4E70037F01227E1835
:1034EF007FDF123A83EF4E600C1242DAEF24D024C2
:1034FF00FF920F8002D20F7E187FE5123A83EF4EB4
:10350F00600C1242DAEF24D0906681F08005E490CF
:10351F006681F07E187FEB123A83EF4E600C1242F9
:10352F00DAEF24D090668DF08005E490668DF07E02
:10353F00187FF1123A83EF4E600C1242DAEF24D06B
:10354F0024FF92018002C20190633E63A201906644
:10355F007B63A2017F0612266E30013B7E187FF738
:10356F00123A83EF4E603012000390667BEFF01239
:10357F00000390667CEFF012000390667DEFF0126F
:10358F00000390667EEFF012000390667FEFF0125B
:0A359F000003906680EFF07F002229
:10411600906576E0C3947C40027F0A906576E0FE67
:1041260004F074B42EF582E43462F583EFF0BF0A2E
:1041360027906576E0FF04F074B42FF582E43462CC
:10414600F583E4F0906576E0FF123B08906576749F
:0941560008F09062B5E004F022CB
:1040BC009080007480F090633663A201F583F582E2
:1040CC0063A2017F0812266E90633E63A20190806A
:1040DC008863A2017F0A12266E9080927407F0A367
:1040EC0074D0F0A37406F0906348E0FF9080B1F0B8
:1040FC009080E1EFF09080957455F0A3F0908000E3
:0A410C007401F090800974F0F022B5
:103E0600908009E04410F09080A0E070609080A15E
:103E16007482F09080A874FFF0A3F0A3F0A3F07F63
:103E2600039080AEEFF0A374CBF09080007402F0A4
:103E3600906B5312224D00000000906B53E090806F
:103E460040F0906B54E0908041F0906B55E090808C
:103E560042F0906B56E0908043F0A3E4F0A3F0A309
:0D3E6600F0A3F0908018F0A3F0A3F0A3F0FB
:013E7300222C
:10406000908009E04440F09080D17482F07F03900A
:1040700080DEEFF0A374CCF09080027402F0906BBD
:104080005712224D00000000906B57E0908058F0CE
:10409000906B58E0908059F0906B59E090805AF006
:1040A000906B5AE090805BF0A3E4F0A3F0A3F0A340
:0B40B000F0908030F0A3F0A3F0A3F02C
:0140BB0022E2
:103D1400908009E04420F09080B8E0706C9080B905
:103D24007482F07F039080C6EFF07FCDA3EFF07F25
:103D3400039080C4EFF0A374CDF09080C074FFF0C2
:103D4400A3F0A3F0A3F09080017402F0906B5B12D7
:103D5400224D00000000906B5BE090804CF0906B73
:103D64005CE090804DF0906B5DE090804EF0906B45
:103D74005EE090804FF0A3E4F0A3F0A3F0A3F090F2
:093D84008024F0A3F0A3F0A3F0E9
:013D8D002213
:103C12008C488D49A907EAFDE975F018A424ACFF88
:103C2200E5F034808F82F583EDF0EBFDE975F01855
:103C3200A4FFAEF024ACFBEE34808B82F583A3EDBF
:103C4200F08549828C83E0FDEF24A8FFEE3480FEEC
:103C52008F82F583EDF08549828C83A3E08F828E7B
:103C620083A3F0854982854883A3A3E0FDE975F02B
:103C720018A424A8FFE5F03480FE8F82F583A3A365
:103C8200EDF08549828C83A3A3A3E08F828E83A368
:043C9200A3A3F022D6
:063975008D4DAB07AA0610
:10397B00908000E030E5079065787401F022906B41
:10398B0053E0FCA3E0FDA3E0FEA3E0F5518E508DC8
:10399B004F8C4EAE02AF038E838F8263A201E55034
:1039AB00540744C0F58385518263A201AF4D1226A3
:1039BB00E0E4FCFDFEE551254DF551EE3550F5509B
:1039CB00ED354FF54FEC354EF54E908040E54EF012
:1039DB00A3E54FF0A3E550F0A3E551F09080007400
:1039EB0020F0AF51AE50AD4FAC4E906B5312224105
:0139FB0022A9
:0639FC008D48AB07AA068E
:103A0200908002E030E5079065787403F022906BB5
:103A120057E0FCA3E0FDA3E0FEA3E0F54C8E4B8D46
:103A22004A8C49AE02AF038E838F8263A201E54BBB
:103A3200540744D0F583854C8263A201AF48122615
:103A4200E0E4FCFDFEE54C2548F54CEE354BF54B2C
:103A5200ED354AF54AEC3549F549908058E549F08B
:103A6200A3E54AF0A3E54BF0A3E54CF09080027485
:103A720020F0AF4CAE4BAD4AAC49906B571222418D
:013A82002221
:02371B008F48D5
:10371D00908001E030E5099065787402F07F002219
:10372D00906B5BE0FCA3E0FDA3E0FEA3E0F54C8E07
:10373D004B8D4A8C4990667B63A201E54B5407443F
:10374D00C8F583854C8263A2017F061226F6E54CEF
:10375D002406F54CE4354BF54BE4354AF54AE43592
:10376D0049F54990657963A201E54B540744C8F5C5
:10377D0083854C8263A201AF481226F6E4FCFDFE60
:10378D00E54C2548F54CEE354BF54BED354AF54AF4
:10379D00EC3549F54990804CE549F0A3E54AF0A395
:1037AD00E54BF0A3E54CF09080017420F0AF4CAEEA
:0D37BD004BAD4AAC49906B5B122241AF4806
:0137CA0022DC
:102F6B009081E0E0F54805480548054805480548C7
:102F7B0005480548054805480548908010E0F54B85
:102F8B00A3E0F54CA3E0F54DA3E0F54E9081E1E015
:102F9B00F5480548054805480548054805480548CE
:102FAB00054805480548908014E0F54FA3E0F5501F
:102FBB00A3E0F551A3E0F552E551B54D08E552B547
:102FCB004E037F0022E4F548E551540744E0F583B6
:102FDB0085528263A20190637563A2017F08122759
:102FEB002690637763A2019062AE63A2017F061203
:102FFB00266E906375E0F549A3E0F54AE4F5489039
:10300B006375E0702AA3E024F8F548E551540744B2
:10301B00E0F58385528274082582F582E43583F5C9
:10302B008363A20190637563A201AF48122726AE9A
:10303B0049E4FCFDE552254AF552E5513EF551EDCB
:10304B003550F550EC354FF54F908014E54FF0A30C
:10305B00E550F0A3E551F0A3E552F09080007440E9
:03306B00F0AF487B
:01306E00223F
:102920009081E6E0F5480548054805480548054812
:1029300005480548054805480548908028E0F54BBE
:10294000A3E0F54CA3E0F54DA3E0F54E9081E7E060
:10295000F54805480548054805480548054805481F
:1029600005480548054890802CE0F54FA3E0F55058
:10297000A3E0F551A3E0F552E4F548E551B54D0A61
:10298000E552B54E05C208022A8CE551540744F0C1
:10299000F58385528263A20190637563A2017F086B
:1029A000122726906375E0F549A3E0F54AE54A450C
:1029B0004970099080027410F07F0022906682E0D6
:1029C000FFF46030906377E06F6003022A539066F3
:1029D00083E0FF906378E06F7079906684E0FF9009
:1029E0006379E06F706D906685E0FF90637AE06FC9
:1029F0006031805F906377E0906682F0906378E06A
:102A0000906683F0906379E0906684F090637AE05A
:102A1000906685F090637BE0FFA3E0906349CFF080
:102A2000A3EFF0906375E0702AA3E024F8F548E581
:102A300051540744F0F58385528274082582F5824B
:102A4000E43583F58363A20190637563A201AF4807
:102A5000122726AE49E4FCFDE552254AF552E55120
:102A60003EF551ED3550F550EC354FF54FAF4EAECC
:102A70004DAD4CAC4BAB52AA51A950A84FD312222A
:102A80003040099080027410F07F002290802CE585
:102A90004FF0A3E550F0A3E551F0A3E552F090808C
:062AA000027440F0AF4893
:012AA600220D
:102AA7009081E3E0F548054805480548054805488D
:102AB7000548054805480548054890801CE0F54B42
:102AC700A3E0F54CA3E0F54DA3E0F54E9081E4E0DB
:102AD700F548054805480548054805480548054897
:102AE700054805480548908020E0F54FA3E0F550DC
:102AF700A3E0F551A3E0F552E4F548E551B54D0AD9
:102B0700E552B54E05C209022BFDE551540744E8CD
:102B1700F58385528263A20190600463A2017F0E50
:102B270012273C906004E0F549A3E0F54A90600C59
:102B3700E0FFF4604A90667BE0FEEF6E7079A3E0F9
:102B4700FF90600DE06F706F90667DE0FF90600E04
:102B5700E06F706390667EE0FF90600FE06F7057E4
:102B670090667FE0FF906010E06F704B906680E0AA
:102B7700FF906011E06F703FE4906013F080089061
:102B8700601374FFF0D2D9906004E0702AA3E024A8
:102B9700F2F548E551540744E8F583855282740EEF
:102BA7002582F582E43583F58363A201906004638F
:102BB700A201AF4812273CAE49E4FCFDE552254A85
:102BC700F552E5513EF551ED3550F550EC354FF5E1
:102BD7004FAF4EAE4DAD4CAC4BAB52AA51A950A81E
:102BE7004FD31222305006E54A45497009908001BB
:102BF7007410F07F0022908020E54FF0A3E550F09D
:102C0700A3E551F0A3E552F09080017440F0AF487E
:012C1700229A
:04315F008E4D8F4EB4
:10316300908000E030E5079065787401F022906B61
:1031730053E0FCA3E0FDA3E0FEA3E0F5548E538DE2
:10318300528C51E554FFE5535407FEE42FF550EEFE
:1031930034C0F54F855082F5837423F00550E55014
:1031A3007002054F534FC7F582854F83740AF005AC
:1031B30050E5507002054F534FC790633E63A20121
:1031C300854F8385508263A2017F061226E0740631
:1031D3002550F550E4354FF54F854D83854E826379
:1031E300A201854F8385508263A2011226C4E4FCA9
:1031F300FDFE906B53E0F8A3E0F9A3E0FAA3E02F00
:10320300FFEE3AFEED39FDEC38FCEF2408FFE43E17
:10321300FEE43DFDE43CFC906B53122241906B5362
:10322300E0908040F0906B54E0908041F0906B55BB
:10323300E0908042F0906B56E0908043F0908000E5
:033243007420F004
:013246002265
:0A2E64008E4D8F4E8C4F8D508B5118
:102E6E00908000E030E5079065787401F022906B59
:102E7E0053E0FCA3E0FDA3E0FEA3E0F5578E568DD4
:102E8E00558C54E557FFE5565407FEE42FF553EEE7
:102E9E0034C0F552855382F5837423F00553E55300
:102EAE00700205525352C7F582855283740AF0059B
:102EBE0053E553700205525352C790633E63A2010D
:102ECE0085528385538263A2017F061226E0740623
:102EDE002553F553E43552F552854D83854E826365
:102EEE00A20185528385538263A2011226C48F5894
:102EFE00EF2553F553E43552F552E5516017854FE2
:102F0E008385508263A20185528385538263A20119
:102F1E00AF511226E0E55824082551F551FFE4FC87
:102F2E00FDFEE5572FF557EE3556F556ED3555F5B1
:102F3E0055EC3554F554908040E554F0A3E555F02A
:102F4E00A3E556F0A3E557F09080007420F0AF573C
:0C2F5E00AE56AD55AC54906B531222419E
:012F6A002244
:063404008E498F4A8D4B3A
:10340A00908000E030E5079065787401F022906BB7
:10341A0053E0FCA3E0FDA3E0FEA3E0F5518E508D3E
:10342A004F8C4EE551FFE5505407FEE42FF54DEE63
:10343A0034C0F54C854D82F5837423F0054DE54D76
:10344A007002054C534CC7F582854C83EBF0054D51
:10345A00E54D7002054C534CC790633E63A201854B
:10346A004C83854D8263A2017F061226E0740625ED
:10347A004DF54DE4354CF54C854983854A8263A266
:10348A0001854C83854D8263A201AF4B1226E074FD
:10349A0008254BF54BFFE4FCFDFEE5512FF551EEF7
:1034AA003550F550ED354FF54FEC354EF54E9080D1
:1034BA0040E54EF0A3E54FF0A3E550F0A3E551F047
:1034CA009080007420F0AF51AE50AD4FAC4E906B6F
:0434DA005312224126
:0134DE0022CB
:023B08008F61CB
:103B0A00908000E030E5079065787401F022906BB0
:103B1A0053E0FCA3E0FDA3E0FEA3E0F5658E648D0F
:103B2A00638C62E565FFE5645407FEE42FFFEE341B
:103B3A00C09062B463A201F5838F8263A201AF6170
:103B4A001226E0E4FCFDFEE5652561F565EE3564C7
:103B5A00F564ED3563F563EC3562F562908040E516
:103B6A0062F0A3E563F0A3E564F0A3E565F0908055
:103B7A00007420F0AF65AE64AD63AC62906B531213
:023B8A002241D6
:013B8C002216
:063247008E4B8F4CAB051D
:10324D00908000E030E5079065787401F022906B76
:10325D0053E0FCA3E0FDA3E0FEA3E0F5528E518DFB
:10326D00508C4FE552FFE5515407FEE42FF54EEE1D
:10327D0034C0F54D854E82F5837423F0054EE54E31
:10328D007002054D534DC7F582854D83EBF0054E0C
:10329D00E54E7002054D90633E63A201854D838519
:1032AD004E8263A2017F061226E07406254EF54E6E
:1032BD00E4354DF54D534DC7E54B854E82854D8318
:1032CD00F0054EE54E7002054D534DC7F582854D07
:1032DD0083E54CF0054EE54E7002054D534DC7E5A7
:1032ED0052240AF552E43551F551E43550F550E4C8
:1032FD00354FF54F908040E54FF0A3E550F0A3E535
:10330D0051F0A3E552F09080007420F0AF52AE5111
:0A331D00AD50AC4F906B53122241EB
:013327002283
:103EDD00908009E04480F09080E97441F07F099072
:103EED0080F6EFF0A37464F09080037402F090807C
:103EFD0003E020E1F9906A4F12224D00000000907E
:103F0D006A4FE0908064F0906A50E0908065F09088
:103F1D006A51E0908066F0906A52E0908067F0A35D
:103F2D00E4F0A3F0A3F0A3F090803CF0A3F0A3F095
:023F3D00A3F0EF
:013F3F00225F
:103328009081E9E0F54905490549054905490549F7
:1033380005490549054905490549908034E0F54A9C
:10334800A3E0F54BA3E0F54CA3E0F54D9081EAE04E
:10335800F549054905490549054905490549054905
:10336800054905490549908038E0F54EA3E0F54F39
:10337800A3E0F550A3E0F551E550B54C08E551B58B
:103388004D037F0022AF51AE50AD4FAC4EAB4DAAAE
:103398004CA94BA84AD3122230400AAF51AE4DEE89
:1033A8009FF549800AAF51EFF404AE4D2EF549E57B
:1033B80050540744E0F58385518263A201906A5313
:1033C80063A201AF49122754E4FCFDFEE5512549EB
:1033D800F551EE3550F550ED354FF54FEC354EF5CE
:1033E8004E908038E54EF0A3E54FF0A3E550F0A3EA
:0B33F800E551F09080037440F0AF49F5
:0134030022A6
:02306F008F4987
:103071009080E8E0640660037FFF22906A4FE0FCE5
:10308100A3E0FDA3E0FEA3E0F54D8E4C8D4B8C4AF1
:10309100E4FFFEFDFCAB4DAA4CA94BA84AC312228A
:1030A1003070609081F9E0F54A906A4FE0FCA3E04E
:1030B100FDA3E0FEA3E0FFE4FAF9F8EF2401FFEA43
:1030C1003EFEE93DFDE83CFC906A4F122241906AC8
:1030D1004FE0FCA3E0FDA3E0FEA3E0FFE4F8EF2452
:1030E10001FFEA3EFEE93DFDE83CFC906A4F1222F9
:1030F10041908064E0F54AA3E0F54BA3E0F54CA3D1
:10310100E0F54D906A5363A201E54C540744D8F5AC
:1031110083854D8263A201AF4912270EE4FCFDFEB7
:10312100E54D2549F54DEE354CF54CED354BF54B5F
:10313100EC354AF54A908064E54AF0A3E54BF0A3EB
:10314100E54CF0A3E54DF09080037420F0AF4DAE57
:0D3151004CAD4BAC4A906A4F1222417F00FA
:01315E00224E
:1042A000A2AF9210C2AF438E2075D2028F828E834E
:0C42B000E0FFE4F5D2538EDFA21092AFC5
:0142BC0022DF
:10423400E5D220E0FBA2AF9210C2AF43D2028F823C
:104244008E83EDF075D25063D250A21092AFE5D2B6
:0342540020E0FB6C
:014257002244
:103C9600E4FDED2401FFE433FE1242A074362DF557
:103CA60082E43463F583EFF00DBD3FE6E4FDED24D9
:103CB6007FFFE433FE1242A0742D2DF582E43461B9
:103CC600F583EFF0742D2DF582E43461F583E07011
:103CD6001B742D2DF582E43461F5837420F0742E67
:103CE6002DF582E43461F583E4F080040DBD80BED9
:103CF600E49061ACF0FDEDFF7E001242A074AD2DA4
:0D3D0600F582E43461F583EFF00DBDFEE9B8
:013D1300228D
:0241DA008B4D0B
:1041DC00A2AF9210C2AF85A24E53A2FE8E838F82E5
:1041EC0005A28C838D82740912276AE54D53A2FEB9
:1041FC0043A22012276C53A2DF854EA2A21092AFCD
:01420C00FFB2
:01420D00228E
:1042BD00A2AF9210C2AF8C838D82EF12276A43A2F8
:0C42CD002012276C53A2DFA21092AFFF5A
:0142D90022C2
:024258008F488D
:10425A00A2AF9210C2AFE4F5838D82740612276A68
:10426A00E54843A22012276C53A2DFA21092AF7F27
:01427A000142
:01427B002220
:02427C008F4869
:10427E00A2AF9210C2AFE4F5838D82740A12276A40
:10428E00E54843A22012276C53A2DFA21092AF7F03
:01429E00011E
:01429F0022FC
:10259300A907E7FFA805EF93C3966008403B74FCC7
:1025A3002FFF80F00F08EF93C3966008402B74FB56
:1025B3002FFF80E00F08EF93C3966008401B74FA67
:1025C3002FFF80D00F08EF93D3966008400B74F968
:1025D3002FFF80C01F1F1F1F1FEF54FEF80303F7B9
:1025E300E893FC08E893FD08E893FE08E893FF22CC
:1025F30009E993C39D6008402974FB29F980F10917
:10260300E993C39E6008401A74FA29F980E209E944
:1026130093D39F6008400B74F929F980D3191919D2
:102623001919E9C313C313FF22740093F8ECC39879
:102633004024701F740193F8EDC39840197014740B
:0E2643000293F8EEC398400E7009740393F8EA
:10265100EFC39840037F00227F0122EDF8E6F008E6
:10266100A3DFFA22EDF8E0F608A3DFFA22E0A36384
:10267100A201F0A363A201DFF475A2002263A2010B
:10268100F0A363A20122E0A363A201F0A363A2016C
:10269100E0A363A201F0A363A201E463A201F0A39A
:1026A10063A201DFE175A20022E0A363A2016DFE36
:1026B100936CFDEE058393FC158363A201DFEA753C
:1026C100A200227F00E493A363A201F00F600CA398
:1026D100E583C2E3F58363A20180EA75A20022E0EB
:1026E100A363A201F0A3E583C2E3F58363A201DF43
:1026F100EE75A20022E0A363A201F0A3E583C2E488
:10270100D2E3F58363A201DFEC75A20022E0A363AB
:10271100A201F0A3E58344F8C2E5F58363A201DFDA
:10272100EC75A20022E583C2E3F583E0A363A20175
:10273100F0A363A201DFEE75A20022E583C2E4D219
:0A274100E3F583E0A363A201F0A317
:10274B0063A201DFEC75A20022E58344F8F583E078
:10275B00A363A201F0A363A201DFEE75A20022F92D
:10276B0022C002C004C00612FFF0D006D004D00273
:01277B00223B
:10234B003E2A2C312CCFE0F0E0ECE5F2F0FB20F84C
:10235B00E8EDFB2043414E0A003E4C2C6B30312CF8
:10236B0025732C43EAEEF0EEF1F2FC20EDE020F8C1
:10237B00E8EDE52043414E2C30202D20353030EA5E
:10238B00E1283530EC292C31202D203530EAE1289D
:10239B00353030EC290A0030202D20353030EAE181
:1023AB00283530EC290031202D203530EAE1283555
:1023BB003030EC29003E2A2C312CCFE0F0E0ECE55C
:1023CB00F2F0FB20EFF0EEF2EEEAEEEBE0204654FB
:1023DB00330A003E4C2C4930312C256C752CD1EA3C
:1023EB00EEF0EEF1F2FC20EEE1ECE5EDE02C31321B
:1023FB0030302C323430302C343830302C393630BD
:10240B00302C31393230300A003E532C4931322CCA
:10241B002562752CC0E4F0E5F120E1EBEEEAE0205B
:10242B00D2C8D220EDE020F8E8EDE50A003E532CAF
:10243B006D2562752C25732CCFF0E8E1EEF020258D
:10244B0062752028C0E4F0E5F120E820EFE0F0E031
:10245B00ECE5F2F0FB290A003E532C5630382C25C4
:10246B00752CCFE0F3E7E020E220EEEFF0EEF1E0A9
:10247B00F528ECF1290A003C6B30313D003C49302A
:10248B00313D003C4931323D003C5630383D002057
:10249B0043616E457247495400200A002043616E28
:1024AB00457272434821000A000A5265713A00498D
:1024BB006E69745443500A004C697374656E5443CF
:1024CB00500A00534F434B5F5443505F45535441A5
:1024DB00424C49534845440A000A2D3E20000A3C11
:1024EB002D2000203C20000ACEF8E8E1EAE020CACB
:1024FB00D13121000ACEF8E8E1EAE020CAD132213D
:10250B00000A455252210A003C6D303D000000008C
:10251B003C6D313D000000003C6D323D0000000081
:10252B003C6D333D000000003C6D343D000000006D
:10253B003C6D353D000000003C6D363D0000000059
:10254B003C6D373D000000003C6D383D0000000045
:10255B003C6D393D000000003C6D31303D0000000A
:10256B003C6D31313D0000003C6D31323D000000CF
:10257B003C6D31333D0000003C6D31343D000000BB
:08258B003C6D31353D000000FC
:0100210022BC
:03002300023B8D10
:0B3B8D00C0E0C083C082C0D075D0181B
:103B9800309840E5E92423F5EB30D707E5F904F53B
:103BA800FB800385F9FBD291AF99C298E537701471
:103BB800BF0520742B2537F582E43469F583EFF0CF
:103BC8000537800F742B2537F582E43469F583EFC8
:103BD800F0053730992BE53CC395365013AE3C05BC
:103BE8003C742B2EF582E4346AF583E0F599800F56
:103BF800E53CC395364008053CD296C290C219C22E
:013C08009922
:093C0900D0D0D082D083D0E0328B
:102C18007BFF7A23794B121D6990688FE0701475D9
:102C280050FF7551237552A27BFF7A237964121DD8
:102C38006980127550FF7551237552B17BFF7A2355
:102C48007964121D697BFF7A2379C0121D69906A25
:102C58004DE0FEA3E0FFC3E49FFFE49EFEAB07FA4E
:102C68003395E0F9F87F007E8C7D0A7C0012219074
:102C78008F538E528D518C507BFF7A2379DE121D33
:102C8800697BFF7A247914906890E0F550121D69E9
:102C9800E4906B5FF0906B5FE0FFC36480949040BA
:102CA80003022D3A90689A7420F0E4A3F0EF33956C
:102CB800E0FEEF7803C333CE33CED8F92413F58280
:102CC80074253EAF82FE123A83EF4E6041E4906B6A
:102CD80061F01242DA906B60EFF0643C601BE0FF39
:102CE800A3E0FE04F0EEFD3395E0FC749A2DF58226
:102CF80074683CF583EFF080D9906B61E0FF339501
:102D0800E0FE749A2FF58274683EF583E4F0906BC8
:102D18005FE0F55075510175526875539A04F55482
:102D28007BFF7A247938121D69906B5FE004F0020A
:102D38002C9D906A4BE0FEA3E0FF7C007D0A1220E8
:0E2D4800B08E508F517BFF7A247963121D6983
:012D5600225A
:063F4000AB07AA06A9056B
:103F4600E4F540F541AF0119EF60458B828A83E0C5
:103F5600FDE4FCED5480FEE4EE6240E54030E716F9
:103F6600E54125E0F541E54033F540434101634134
:103F7600B263409E800BE54125E0F541E54033F50F
:103F860040ED25E0FD0CBC08CA0BBB00010A80B55C
:0C3F9600E540906899F09068EAE541F081
:013FA20022FC
:1018FD00E4F540F541854182854083E4F00541E5FD
:10190D004170020540B400EDE540B404E8E4906890
:10191D008FF07E247F82123A83EF4E601B1242DAE3
:10192D008F48E548B4310690688F740AF0E548B4E5
:10193D00320690688F7464F07E247F88123A83EFAC
:10194D004E6023124003A804A905AA06AB077F0029
:10195D007E8C7D0A7C00122190122222906A4DEE1F
:10196D00F0A3EFF0800A906A4D74FFF0A374B8F005
:10197D007E247F8E123A83EF4E600A1240039068E8
:10198D0090EFF08005E4906890F07E247F94123AF9
:10199D0083EF4E6016124003E47B0AFAF9F8122128
:1019AD0005906A4BEEF0A3EFF08009906A4BE4F0DE
:1019BD00A37464F0E4F549F543F544F548AF48EFF9
:1019CD003395E0FEEF7803C333CE33CED8F924132D
:1019DD00F58274253EAF82FE123A83EF4E700302FC
:1019ED001CF21240038F45E5457003021D00E545CD
:1019FD00B4FF03E4F545854482854383A37405F064
:101A0D00854482854383A3A37464F0854482854312
:101A1D0083A3A3A3E4F0E5442404F582E43543F560
:101A2D0083E4F0E5442405F582E43543F583E5458B
:101A3D00F0E5442406F582E43543F583E4F0E5440E
:101A4D002407F582E43543F5837407F0E544240853
:101A5D00F582E43543F5837438F0E5442409F582C5
:101A6D00E43543F583E4F0E544240AF582E4354397
:101A7D00F583E4F0E544240BF582E43543F583E486
:101A8D00F0E544240CF582E43543F583E4F0E544B8
:101A9D00240DF582E43543F583E4F0E544240EF599
:101AAD0082E43543F583E4F0E544240FF582E43513
:101ABD0043F583E4F0E5442410F582E43543F583E2
:101ACD00E4F0E5442403FFE43543FE7D0E123F4070
:101ADD00906899E0FFE5442411F582E43543F583E0
:101AED00EFF09068EAE0FFE5442412F582E4354317
:101AFD00F583EFF08544828543837412F0E58224EB
:101B0D001AF582E43583F583E4F0AA43A9447B01F9
:101B1D008B338A34893590001FE54912208E900051
:101B2D001DE412208E74202544F544E43543F5431D
:101B3D00906898E004F01242DAEF12227E1CF20057
:101B4D001CF2211B84231CF23C1C1A431C32461B25
:101B5D00A3491BD2501BEA511C02531BBA551CD66C
:101B6D00631C32661C4A691C82701C9E711CBA7300
:101B7D001C667500001B431242DA75F008EFA424B1
:101B8D008BF582E5F03423AF82FE123A83EF4E607F
:101B9D00A512400380A0AB33E535241BF9E43534A1
:101BAD00FA122063440112207C05498089AB33E58C
:101BBD0035241BF9E43534FA122063440212207CDB
:101BCD000549021B43AB33E535241BF9E43534FAE3
:101BDD00122063440412207C0549021B43AB33E5FC
:101BED0035241BF9E43534FA122063440812207CA5
:101BFD000549021B43AB33E535241BF9E43534FAB3
:101C0D00122063441012207C0549021B43AB33E5BF
:101C1D0035241BF9E43534FA122063442012207C5C
:101C2D000549021B43AB33E535241BF9E43534FA82
:101C3D00122063444012207C0549021B43AB33E55F
:101C4D0035241CF9E43534FA122063440112207C4A
:101C5D0074032549F549021B43AB33E535241CF9C3
:101C6D00E43534FA122063440212207C74032549B2
:101C7D00F549021B43AB33E535241CF9E43534FA41
:101C8D00122063440412207C74032549F549021B7C
:101C9D0043AB33E535241CF9E43534FA12206344A3
:101CAD000812207C74032549F549021B43AB33E52B
:101CBD0035241CF9E43534FA122063441012207CCB
:101CCD0074032549F549021B43AB33E535241CF953
:101CDD00E43534FA122063442012207C7403254924
:101CED00F549021B430548C3E548648094905003B1
:091CFD000219CAE4F543F544FFA5
:011D060022BA
:10420E00C2A9438902758C48758A4875D90475DB35
:10421E004875DC4875DD4875DE48E4F5E9F5F9C208
:06422E00D9D28CD2DE2281
:103E740043AB01C2E8C2EAE4FFEFC454F0F5B1C3B6
:103E8400EF64809488500575B3D08003E4F5B3E4FF
:103E9400F5B275BCC8F5BDF5BE75BF7875C4FFF540
:103EA400C5F5C675C778F5A3F5A3F5A3F5A3F5A3E2
:103EB400F5A3F5A3F5A30FBF0EBF90688FE0FF2510
:103EC400E0F5B475B50C75B66C75A11275AB0275D9
:083ED400C13E75C3FF75C20376
:013EDC0022C3
:103FA30075B180E4F5B3F5B28526BCE5275403FF6C
:103FB30033333354F8FFE52754E04FFFE528C413A8
:103FC30054074FF5BDE52833333354F8FFE529C4CF
:103FD3001354074FF5BEE52933333354F8F5BF8542
:103FE3002BA3852CA3852DA3852EA3852FA38530F5
:103FF300A38531A38532A3E52A540F2450F5B322B8
:102D5700E59B541F6020200B1A7E247F9A12315F57
:102D6700E59B541FFF7E007D031232477E247FA41C
:102D770012315FE4F59BE5BA30E008E4F5B375B1CD
:102D870080F5B2E5CFF47003022E61754A01E4F5D0
:102D970049E5CFF4554A7003022E4FE549C454F074
:102DA700F5B1E5B2547F6420706FE5B3540FF52A8F
:102DB70085BC26E5BD541FFF131313541FFFE5BD44
:102DC70054E044184FF527E5BDC43354E0FFE5BE92
:102DD700131313541F4FF528E5BEC43354E0FFE522
:102DE700BF131313541F4FF52985A32B85A32C85D8
:102DF700A32D85A32E85A32F85A33085A33185A376
:102E070032E4F5B2E526547EB5260575B350800346
:102E170075B3D0E52A2405FF22E5B2549F6023202D
:102E27000B207E247FA712315FAFB27E007D031295
:102E37003247AFB37E007D031232477E247FB21242
:102E4700315FE4F5B275B3D0E54A25E0F54A0549A7
:0C2E5700E549C394085003022D987F0049
:012E6300224C
:10366800C219E4F537F50BD296F536F53CF524FF8B
:103678007F409068EBE4F0A3DFFCE4906896F0A349
:10368800F0FF75F002EFA4248FF582E5F03466F5BB
:103698008374FFF075F002EFA42490F582E5F0340E
:1036A80066F583747FF00FBFFED8E4906896F0A3A8
:1036B800F0F53DF5461218FD123E74C2ADE4F5C9A9
:1036C800D2CDD2CCC2C9C2CAF5CDF5CC906A4DE0F4
:1036D800F5CBA3E0F5CA85CBCD85CACCE4F59853E4
:1036E80087BFD29E438740C29FC2ACC298C2997519
:1036F800B81075B710D2CAD29CD2AC12420EC2D939
:10370800E5E92464F5EB30D706E5F904F5FB2285F5
:02371800F9FBBB
:01371A00228C
:0100220022BB
:01430B00228F
:01430C00228E
:01430D00228D
:103D8E00854482854383E07010F543F54485448273
:103D9E00854383E070037F0122E5442401FFE4356F
:103DAE0043F5838F8263A201906A2B63A2017F1475
:103DBE0012266E854482854383E0F536E5444543FD
:103DCE00700B052453240F906896F0A3F0200B0778
:103DDE007E247FB412315FE4F53CD290C291C2963C
:103DEE00C2992099FDD299200B0B7E6A7F2BE4FBA2
:083DFE00AD361234047F0022EF
:10385B00E546C394404003E4F54674EB2546F582F8
:10386B00E43468F583E0FF30E16F74EB2546F582B5
:10387B00E43468F583EF54FDF0E4906475F0A374C1
:10388B000DF090667AE0906477F0A37419F0A3744E
:10389B0048F0A37479F0E546131313541FFF906897
:1038AB0090E02F90647BF0E546540725E025E0245B
:1038BB0080A3F0A37408F0F5F0E546A4248FF582FD
:1038CB00E5F03466F58363A20190647E63A2017F09
:0E38DB000812266E05467F012205467F002258
:01430E00228C
:1035A900E4F538F539853F82853E83E0F53A053FF4
:1035B900E53F7002053EF582853E83E0F53B053F18
:1035C900E53F7002053E906896E0FEA3E0248FF582
:1035D9008274663EF583E0653A6029906896E0A3B7
:1035E900E0FF248FF58274663EF583E53AF0EF78C3
:1035F90003CEC313CE13D8F924EBF58274683EF5D4
:10360900837407F0906897E004F07006906896E07C
:1036190004F0906896E0FEA3E0248FF58274663E7C
:10362900F583E0653B6029906896E0A3E0FF248F6D
:10363900F58274663EF583E53BF0EF7803CEC3135C
:10364900CE13D8F924EBF58274683EF5837407F03C
:0F365900906897E004F07006906896E004F02205
:10415F00906896E0FEA3E0248FF58274663EF583A7
:10416F0074FFF0906897E004F07006906896E00492
:10417F00F0906896E0FEA3E0248FF58274663EF51A
:10418F0083747FF0906897E004F07006906896E073
:03419F0004F02207
:100F3F0074EB253DF582E43468F583E020E002058B
:100F4F003DE53DC394404003E4F53D122D57EF605E
:100F5F0069E529640F7063906890E0FF6528705A07
:100F6F0074EB253DF582E43468F583E0FE30E04A0A
:100F7F0074EB253DF582E43468F583EE54FEF0758D
:100F8F002648752779E53D131313541FFEEF2EF5F1
:100F9F0028E53D540725E025E02480F529752A082A
:100FAF0075F008E53DA4248FF582E5F03466F583EE
:100FBF007D2B7F08122665123FA3300249C2029093
:100FCF006892E004F07006906891E004F0D39068A6
:100FDF0092E094B8906891E0940B402AE4F0A3F06B
:100FEF00F54874EB2548F582E43468F583E030E288
:100FFF000E74EB2548F582E43468F5837407F00529
:10100F0048E548B440DC3000469080E8E0700F12AD
:10101F003EDD300D077E247FBA12315FC21D9080F6
:10102F00E8E0B40E129080037408F0300D077E24B0
:10103F007FC312315FC21D9080E8E0B4060F201D00
:10104F000C300D077E247FCE12315FD21DC20020DF
:10105F001D030211172019071233288F488003E44C
:10106F00F548E5486047300D0C7E247FE47C6A7DAF
:10107F0053FB122E64E5E92410F5EB30D708E5F9A0
:10108F002428F5FB8006E5F92427F5FB906A5363C6
:10109F00A201906A2B63A201AF4812266E854836D3
:1010AF00E4F53CD290C291D219C296D29920D903BD
:1010BF000214A3C2D9E5E92410F5EB30D708E5F9FE
:1010CF002428F5FB8006E5F92427F5FBE537D394B3
:1010DF000050030214A3C291853742E4F53790699B
:1010EF002B63A201906A5363A201AF4212266EAF27
:1010FF004212306F200D030214A37E247FE97C6A15
:10110F007D53AB42122E642220D9030214A3C2D9FD
:10111F00E537D39400500302135EC291853742E442
:10112F00F537F50B200B0D7E247FEE7C697D2B7B35
:10113F0014122E64753E69753F2D053FE53FAE3E97
:10114F007002053E14F5828E83E0641C6003021466
:10115F0099053FE53FAE3E7002053E14F5828E8342
:10116F00E06003021499E5442405F582E43543F564
:10117F0083E0FF053FE53FAC3E7002053E14F5826C
:10118F008C83E06F6003021499053FE53FAE3E701C
:10119F0002053E14F5828E83E060030214997E6986
:1011AF007F2D7D10123F409068EAE0FF906899E034
:1011BF004F6010300B030214997E247FF212315FBF
:1011CF000214997E697F3D7D10123F409068EAE0DE
:1011DF00FF906899E04F6010300B030214997E2442
:1011EF007FFF12315F021499E544241FF582E43525
:1011FF0043F583E075F002A4FF906896E5F0F0A345
:10120F00EFF0E544241DF582E43543F583E4F0E582
:10121F0044241BF582E43543F583E0F54530E009BE
:10122F00753E69753F811235A9E54530E109753E77
:10123F0069753F7F1235A9E54530E209753E69753D
:10124F003F931235A9E54530E309753E69753F9522
:10125F001235A9E54530E409753E69753F9D123594
:10126F00A9E54530E509753E69753F651235A9E574
:10127F004530E609753E69753F671235A9E5442487
:10128F001CF582E43543F583E0F54530E01B753EF0
:10129F0069753F311235A9753E69753F391235A908
:1012AF00753E69753F431235A9E54530E11B753E23
:1012BF0069753F331235A9753E69753F3D1235A9E2
:1012CF00753E69753F451235A9E54530E21B753E00
:1012DF0069753F351235A9753E69753F3F1235A9BE
:1012EF00753E69753F471235A9E54530E31B753EDD
:1012FF0069753F371235A9753E69753F411235A99A
:10130F00753E69753F491235A9E54530E41B753EB9
:10131F0069753F8D1235A9753E69753F8F1235A9D5
:10132F00753E69753F911235A9E54520E503021415
:10133F0040753E69753F5F1235A9753E69753F610E
:10134F001235A9753E69753F631235A9021440E540
:10135F0044241DF582E43543F583E0D3940A50030A
:10136F00021432E544241FF582E43543F583E0751A
:10137F00F002A4FF906896E5F0F0A3EFF0E54424A7
:10138F001BF582E43543F583E0F54530E003124168
:10139F005FE54530E10312415FE54530E20312415D
:1013AF005FE54530E30312415FE54530E403124149
:1013BF005FE54530E50312415FE54530E603124135
:1013CF005FE544241CF582E43543F583E0F54530B1
:1013DF00E00912415F12415F12415FE54530E109BB
:1013EF0012415F12415F12415FE54530E209124140
:1013FF005F12415F12415FE54530E30912415F1211
:10140F00415F12415FE54530E40912415F12415FD0
:10141F0012415FE54530E51912415F12415F1241FC
:10142F005F800EE544241DF582E43543F583E00427
:10143F00F0906A4BE0FEA3E0FF4E6020201B1BE004
:10144F0025E9F5EB30D708EE25F904F5FB80089078
:10145F006A4BE025F9F5FBD21B22C21BE536600B68
:10146F0074202544F544E43543F543E5E924F4F5C8
:10147F00EB30D708E5F92402F5FB8005E5F904F513
:10148F00FB123D8EEF700DC21A22200B077E257FB7
:04149F000C12315F9B
:0114A3002226
:03001E007F00223E
:1038F5000208D0E493A3F8E493A34003F68001F211
:1039050008DFF48029E493A3F85407240CC8C333D3
:10391500C4540F4420C8834004F456800146F6DFA2
:10392500E4800B0102040810204080904304E47EEB
:10393500019360BCA3FF543F30E509541FFEE49397
:10394500A360010ECF54C025E060A840B8E493A35E
:10395500FAE493A3F8E493A3C8C582C8CAC583CA89
:10396500F0A3C8C582C8CAC583CADFE9DEE780BE41
:01430A0000B2
:10206300BB010689828A83E0225002E722BBFE027B
:09207300E32289828A83E49322AE
:10207C00BB010689828A83F0225002F722BBFE0143
:02208C00F3223D
:10208E00F8BB010DE58229F582E5833AF583E8F088
:10209E00225006E92582C8F622BBFE05E92582C834
:0220AE00F2221C
:1020B000BC000BBE0029EF8DF084FFADF022E4CC14
:1020C000F875F008EF2FFFEE33FEEC33FCEE9DECDD
:1020D000984005FCEE9DFE0FD5F0E9E4CEFD22ED23
:1020E000F8F5F0EE8420D21CFEADF075F008EF2F6D
:1020F000FFED33FD4007985006D5F0F222C398FD5E
:052100000FD5F0EA22FA
:10210500E88FF0A4CC8BF0A42CFCE98EF0A42CFC79
:102115008AF0EDA42CFCEA8EF0A4CDA8F08BF0A4F7
:102125002DCC3825F0FDE98FF0A42CCD35F0FCEB56
:102135008EF0A4FEA9F0EB8FF0A4CFC5F02ECD391B
:0F214500FEE43CFCEAA42DCE35F0FDE43CFC2288
:1021540075F008758200EF2FFFEE33FECD33CDCC42
:1021640033CCC58233C5829BED9AEC99E5829840C5
:102174000CF582EE9BFEED9AFDEC99FC0FD5F0D6A2
:10218400E4CEFBE4CDFAE4CCF9A88222B800C1B9CC
:102194000059BA002DEC8BF084CFCECDFCE5F0CB0A
:1021A400F97818EF2FFFEE33FEED33FDEC33FCEB43
:1021B40033FB10D703994004EB99FB0FD8E5E4F9FE
:1021C400FA227818EF2FFFEE33FEED33FDEC33FCEB
:1021D400C933C910D7059BE99A4007EC9BFCE99ADF
:1021E400F90FD8E0E4C9FAE4CCFB2275F010EF2F24
:1021F400FFEE33FEED33FDCC33CCC833C810D70724
:102204009BEC9AE899400AED9BFDEC9AFCE899F85E
:0E2214000FD5F0DAE4CDFBE4CCFAE4C8F922F1
:0E222200C3E49FFFE49EFEE49DFDE49CFC22CD
:10223000EB9FF5F0EA9E42F0E99D42F0E89C45F004
:01224000227B
:0C224100ECF0A3EDF0A3EEF0A3EFF02210
:10224D00A8828583F0D083D0821222641222641278
:10225D002264122264E473E493A3C583C5F0C5839D
:10226D00C8C582C8F0A3C583C5F0C583C8C582C8DB
:01227D00223E
:10227E00D083D082F8E4937012740193700DA3A3EF
:10228E0093F8740193F5828883E473740293686003
:06229E00EFA3A3A380DF03
:101D0700E55C2450F8E6055C22784D3017027850E0
:101D1700E475F0011222D10220632010EB7F2ED24E
:101D2700108018EF540F2490D43440D4FF30140B94
:101D3700EF24BFB41A0050032461FFE55D6002156C
:101D47005D0560E5607002055F30170D784DE4753D
:101D5700F0011222D1EF02207C0241167403D21740
:101D67008003E4C217F55C8B4D8A4E894FE4F55D1D
:101D7700F55FF560E55D60077F20121D4280F57510
:101D87005EFFC211C210C212C213C215C216C21818
:101D9700121D10FF700D3017057F00121D53AF6025
:101DA700AE5F22B4255FC2D5C214121D10FF24D026
:101DB700B40A00501A75F00A785D30D50508B6FFE9
:101DC7000106C6A426F620D5047002D21380D924B2
:101DD700CFB41A00EF5004C2E5D214021F53D21138
:101DE70080C6D21080C0D21280BCD2D580BAD2159C
:101DF70080B47F20121D422012077401B55D004098
:101E0700F1121D07FF121D42021D7BD218D2168048
:101E170095121D07FB121D07FA121D07F94A4B7091
:101E27000679247A207BFF20122EE55D602A7E004A
:101E37008E827583001222A460060EEE655E70F036
:101E4700C2D5EBC0E0EAC0E0E9C0E0EE121F9AD0CD
:101E5700E0F9D0E0FAD0E0FB122063FF60AAEBC004
:101E6700E0EAC0E0E9C0E0121D42D0E02401F9D069
:101E7700E03400FAD0E0FBE55E0460DCD55ED98093
:101E8700877BFF7A1F7996D212809C79108002791E
:101E970008C216C2188008D2D5790A8004790AC206
:101EA700D5E55E047002F55EE4FAFDFEFF121D073C
:101EB700FC7B08201113121D07FD7B1030100A123E
:101EC7001D07FE121D07FF7B20EC3382D592D550EC
:101ED70013C3E43010069FFFE49EFEE42011039D28
:101EE700FDE49CFCE4CBF8C211EC700CCFCECDCC5A
:101EF700E824F8F870F38017C3EF33FFEE33FEEDF5
:101F070033FDEC33FCEB33FB994002FB0FD8E9EBD5
:101F1700301105F8D0E0C448B211C0E00AEC4D4ECC
:101F27004F78207B0070C2EAB55E0040BCC0E0126B
:101F37001F9CD0F0D0E0201104C4C0E0C4B211C08F
:101F4700F0121D2BD0F0D5F0EB021D7B12227E1E66
:101F570018531E92581DE94C1DE5421E964F1E9EB2
:0F1F6700441E9E491DFE431EA4551E88461E881B
:101F7600451E88472044501DED2D1DF12E1E142BA5
:101F86001DF5231E1220202D2A1DAD4800001E0C13
:101F96003F3F3F00790AA2D5201314301509B91026
:101FA600020404B9080104A2D52016025001042037
:101FB60012689212B55D005034C0E07F20301319CC
:101FC6007F30A21272167215500F121FF3C212C280
:101FD60016C215C2187F30800F301503E9C0E01213
:101FE6001D42301503D0E0F9D0E0B55DCC301517B1
:101FF6007F30B9100C121D427F583014077F78804D
:1020060003B90803121D423012057F2D021D427FBF
:10201600202018F87F2B2016F322921280CF286EEC
:10202600756C6C2900D211121D073011F8C2117897
:102036005D30D50108F6021DAD2D50434958121DDD
:10204600072403B405004001E490203F93121D339A
:0D205600743A121D33D213755D04021E9200
:10277C008B4A8A4B894CE4F556F555F554F553F5CF
:10278C0051F552E54E454F454D6012EBC0E0EAC0A5
:10279C00E0E9C0E0AB4DAA4EA94F1222E1AB4A05CD
:1027AC004CE54CAA4B7002054B14F9122063F557FB
:1027BC00C394094007E557D3940D40E1E5576420D5
:1027CC0060DBE557B42D054352038016E557B42B57
:1027DC0005435201800C74FF254CF54C74FF354BAE
:1027EC00F54BE55060046410703FAB4AAA4BA94C02
:1027FC0012206364306009E550702E75500A8029F0
:10280C009000011222A4FF64786004EFB4581343C3
:10281C0052017550107402254CF54CE4354BF54BB8
:10282C008007E5507003755008AB4A054CE54CAA7F
:10283C004B7002054B14F9122063F557C394614099
:10284C000AE557D3947A50035357DF74D02557F5C4
:10285C0057C3940A400CE5579411406D74F92557F1
:10286C00F557E557D39550506043520185565B851B
:10287C00555A855459855358AF507E00E4FCFDAB36
:10288C0056AA55A954A853122105C8ECC8C9EDC9BC
:10289C00CAEECACBEFCBE4FCFDFEEB2557F556EEAA
:1028AC003AF555ED39F554EC38F553AF56AE55AD08
:1028BC0054FCAB5BAA5AA959A858D3122230500326
:1028CC00022835435204022835E55220E003E48007
:1028DC002DE54E454F454D601EAB4AE54C24FFF9A6
:1028EC00E54B34FFFAEBC0E0EAC0E0E9C0E0AB4DE9
:1028FC00AA4EA94F1222E1E55230E20774FFFFFE07
:10290C00FDFC22E552AF56AE55AD54AC5330E1034D
:04291C00022222224F
:1022A400BB010CE58229F582E5833AF583E02250EF
:1022B40006E92582F8E622BBFE06E92582F8E22239
:0D22C400E58229F582E5833AF583E4932253
:1022D100FAE6FB0808E6F925F0F618E6CA3AF6220E
:1022E100BB011A89828A83D0F0D0E0F8D0E0F9D01E
:1022F100E0FAD0E0FBE8C0E0C0F00223395016E973
:10230100F8D083D082D0E0F9D0E0FAD0E0FBC082EF
:10231100C083022330BBFE16E9F8D083D082D0E01F
:0F232100F9D0E0FAD0E0FBC082C0830223422251
:09233000EBF608EAF608E9F622D2
:09233900EBF0A3EAF0A3E9F022A5
:09234200EBF208EAF208E9F222CC
:00000001FF
